:10000000E20141084B0849085008490843082D08F7
:10001000500847084D08560835082E0833083008A0
:100020000D0868001E091E091E091E091E091E0969
:100030001E091E091E091E09E802120A0008100CFA
:1000400029001504F60405050000360335030307EF
:10005000C6040306C6050307F6040306F6050000FA
:100060000000000005040000000000000000E9029C
:10007000230A0008060C2900050500002E030307CB
:10008000C6040306C60500000000000005040000C9
:1000900000000000E9023C0A0008FF0C0600000016
:1000A00000000000100C2900050500000000000001
:1000B000000000000504C6070304C6060305380354
:1000C0003703E902540ABF0C06001704F8040008BD
:1000D00001022D00380C2C000D02810043066C0A31
:1000E00001022D00100CAC010C0202000E0C2B00C2
:1000F000EB02780A0000080C29001F0C2B00EB0211
:100100007F0A000000000D02810043068D0A0102F3
:100110002D00100CAC010C0202008C0703048C06AD
:1001200003052A03E9027D0A380C02000008E704EF
:10013000210C2B00EB029A0A080C290000002A036C
:1001400000000307E7040306E705210C2B00EB0280
:10015000A70AE9029F0A000000000000000000005A
:100160000000E705200C2B00EB02B40A0008680928
:100170000A02330068090A023200010CB2000307C8
:10018000B3000008100C2C0068000802A304C3048C
:1001900000092A00A304C3049709A304C304A80206
:1001A000EC02C50AF00AF00C2700000C07006500FD
:1001B0006600000C0500000C06000400380C02006C
:1001C00000086500400C2600F20C2700070C050013
:1001D000BF0C06000F0C07000400380C02000008DA
:1001E000A304C304D309400C2A00A304C304970941
:1001F000FE0A380C0200A304C304D309A304C304F9
:100200006809720C8A0043067D0B770C8A0043064E
:10021000B50B620C8A004306620BA305C3058D0B68
:1002200000003F0C8A004306C20AFE0A6809770CE8
:100230008A004306510B720C8A0043063E0B740C75
:100240008A004306240BFE0A6809610C8A004306F3
:10025000320B620C8A004306360B630C8A0043069D
:100260003A0BFE0A68090A020500FE0A68090A023A
:100270000600FE0A68090A020700FE0A6809610C06
:100280008A000307FE0A9C0CCA010306FE0A5C0CE6
:10029000AA000A02240000022A00A304C30497094A
:1002A000FE0A6809610C8A000307FE0A9C0CCA0159
:1002B0000306FE0A5C0CAA000A02240068090A026E
:1002C0002000FE0A6809700C8A004306990B730C23
:1002D0008A0043067A0B640C8A004306740B440CB4
:1002E0008A004306770BFE0AA305C3048C0BA30503
:1002F000C304BA0BA305C304CB0B6809730C8A00B3
:100300004306870B700C8A004306A70BFE0A680998
:10031000A305C304700C8A004306600A640C8A00BB
:100320004306550A630C8A0043064C0AA304C3041F
:10033000FE0A6809A304C3056C0C8A004306660A1A
:10034000730C8A004306330BA304C304FE0A680936
:10035000A304C3056C0C8A004306BD0A730C8A0013
:100360004306F60AA304C304FE0A6809730C8A0054
:100370004306C30B650C8A004306D10B700C8A0040
:100380004306E40BFE0A6809A305C304700C8A0047
:100390004306430B630C8A0043063A0BA304C304D1
:1003A000FE0A6809A305C304650C8A004306B40A63
:1003B000660C8A004306910A630C8A004306AB0A66
:1003C000640C8A0043069E0A6809A305C3056C0CE9
:1003D0008A004306660A730C8A004306270BA304AF
:0403E000C304FE0A4A
:100400006500060C05006600BF0C0600F00C270016
:100410000B0C070000008704140C3F00FF020E0ABB
:10042000C704140C3F00FF02130A8705140C3F0099
:10043000FF02180AA7040008020C2E00A304C3043C
:100440003A09A304C3041F09080C2E00A304C30423
:100450003A09A305C3050009A305C304F102290A4B
:100460000E0C2E00A304C3043A09040C2E003A0912
:10047000A304C3044D09000874006F007900A305AC
:10048000C30400096E00A304C3043A097500760092
:10049000A304C3041F090008A304C304B709A305E8
:1004A000C3043C09A305C304690AA304C304B70930
:1004B000010C3400A305C3040009A305C304690AA1
:1004C000A304C304B7097400A305C3040009A3056A
:1004D000C304040C2E001402EE01A304C3043A0961
:1004E000A304C3044D0938033703F804D8041802E1
:1004F0002A00A304C304970917022A00A304C30413
:100500009709060C2E00A304C3043A09A305C304EB
:10051000010CB2000307B3000306690AA304C30475
:10052000F00AA304C304B70974006F00010C39007A
:10053000A305C3040009A305C304BD0AA304C3049F
:10054000B709010C34006F007900A305C30400094A
:10055000A305C304BD0AA304C304B709A305C304C8
:100560003C09A305C304BD0AA304C304B709790069
:1005700074006F00A305C30400090F022A00A3043E
:10058000C3049709AF02A304C30468090A02360032
:10059000A304C30468090A023500A305C304F606D0
:1005A000140B1907EC0A040C2E001402EE01A3042C
:1005B000C3043A09A304C3044D09A305C3043803C3
:1005C00037031602B8013F0C78014307EC0A150205
:1005D000B7014307EC0A140B020C2E001402EE01C3
:1005E000A304C3043A0975037603A304C3041F09D3
:1005F000080C2E00A304C3043A09A304C304110980
:10060000040C2E001402EE01A304C3043A09A3044F
:10061000C3044D09000000000000000000000000BD
:100620000000000000000000060C2E00A304C3041C
:100630003A09A305C304010CB2000307B300030683
:10064000BD0AA705230B240BC705A304C304F00AA6
:100650002A0C2A00A304C304970918022A00A30441
:10066000C304970917022A00A304C3049709A3052A
:10067000C304210BA304C304B709A305C3043C09A5
:10068000A305C3044C0BA304C304B7097900740089
:100690006F00A305C30400090F022A00A304C304CA
:1006A0009709AF0268090A02360068090A02350094
:1006B000A305C304F606780B750376037000010CDE
:1006C0003100A305C3041C09B002E60CD0010306E7
:1006D000280B1702950043075F0B1802960043078B
:1006E0005F0B100231001002F1011002F1011C0930
:1006F000060C2E00A304C3043A09A305C304010C8D
:10070000B2000307B30003064C0BA705870B880B49
:10071000C705A304C304F00AA305C30400096E00BF
:10072000A304C3043A093F0C3600FF0C35007503DF
:1007300076031F09070C3200060C2E00A304C30425
:100740003A09A305C304F2029C0B010C2E00A3047A
:10075000C3043A09070C2E003A09080C2E003A0986
:100760001109010C2E003A09070C2E003A09A305C5
:10077000C304210BA305C3040009A3046E003A09B6
:100780003F0C3600FF0C35001F09090C2E003A09FA
:100790001109A305210BA304C304B709A305C304CE
:1007A0000009A305C304FF0C3500FF0C3600040C40
:1007B0002E00A304C3043A09A304C3044D0938035B
:1007C0003703F804D8041702750118027601060CE5
:1007D0002E00A304C3043A09A305C304010CB2000C
:1007E0000307B3000306D70B16022A00A304C304B1
:0E07F000970915022A009709A305C304210BDF
:1008000078001A0778041A0678053A0758043A0659
:1008100058055A0738045A0638055B0718045B0662
:10082000180577007B07F7047B06F7059B07D704BD
:100830009B06D7057C07B7047C06B7055C079704C1
:100840005C069705FB077704FB0677053C07570412
:100850003C0657051C0737041C063705BB07170461
:10086000BB06170500087800DB077804DB0678056F
:100870001A0758041A0658053A0738043A06380584
:100880005A0718045A06180577005B07F7045B0639
:10089000F7057B07D7047B06D7059B07B7049B06A4
:1008A000B7057C0797047C0697051C0777041C0690
:1008B0007705BB075704BB0657053B0737043B06C4
:1008C00037051B0717041B0617050008A304C304FC
:1008D000E109A304C304B709A304C305FF0C350051
:1008E000FF0C36006F00C704140C3F00FF02760AAD
:1008F0008704140C3F00FF027B0A65057F0A800A0B
:1009000005023A0006023B0007023C006504A3040E
:10091000C3050009A304C305000C8F0043079F0A09
:1009200018022A00A304C304970917022A00A3048B
:10093000C3049709A304C305010C2F00A30A1702DF
:10094000750118027601A304C305010CB200030768
:10095000B3000306730A8705AD0AAE0AAF0AC705DE
:1009600016022A00A304C304970915022A00A3044F
:10097000C3049709A304C304F00A6300E1096300F8
:10098000B709A304C305C704140C3F00FF02C60A3D
:100990008704140C3F00FF02CB0A6505CF0AD00A7A
:1009A000D10AD20A05023A0006023B0007023C00C7
:1009B0006504A304C305000918022A00A304C304A4
:1009C000970917022A00A304C3049709A304C305C7
:1009D000010CB2000307B3000306C30A8705F00A3F
:1009E000F10AF20AC705A304C304F00AA304C3046E
:1009F000E109090C0700FF0C0600A304C304B709B2
:100A0000A304C305C704140C3F00FF02050BA70491
:100A1000140C3F00FF020A0B65050E0B0F0B0502BD
:100A20003A0006023B0007023C006504A304C3052C
:100A3000330918022A00A304C304970917022A00E5
:100A4000A304C3049709A304C305010CB200030760
:100A5000B3000306020BA7052D0B2E0B2F0BC705AA
:100A6000A304C304F00AA304C304E109090C0700AA
:100A7000FF0C0600A304C304B709A304C305FF0CBD
:100A80003500FF0C36006F00C704140C3F00FF0256
:100A9000470BA704140C3F00FF024C0B6505500BDD
:100AA000510B05023A0006023B0007023C006504B8
:100AB000A304C3053309A304C305000C8F00430737
:100AC000700B18022A00A304C304970917022A0016
:100AD000A304C3049709A304C305010C2F00740BDE
:100AE0001702750118027601A304C305010CB200B8
:100AF0000307B3000306440BA7057E0B7F0B800B97
:100B0000C70516022A00A304C304970915022A0088
:100B1000A304C3049709A304C304F00A2505900B9A
:100B2000910B920B25046300FE0A8605970B980B28
:100B300086046300FE0A6A004505F80C0500A00B58
:100B4000FC0C05002505A40BA50BA60B6A030A04E3
:100B500045060A052504FD029C0BF80C050045041A
:100B600063009709FE0A6A008605B60BB70B6A0395
:100B70000A0446060A058604FD02B40B63009709C1
:100B8000FE0A63006809A304C305080C3D006A035C
:100B9000450403064505CC0BCD0B2505CF0BD00B2B
:100BA000D10B2504FD02C70B4504400C2A0063004D
:100BB0009709FE0A630068090A023D0068090A02F3
:100BC000320068090A023300A304C305100C2A008E
:100BD0001D02AA0073037203EA02EA0B7303720395
:100BE000660403066605F40B8605F60BF70B860410
:100BF000FD02EE0B6604400C2A0063009709FE0A12
:100C0000200C2800E802020A000805023A00060249
:100C10003B0007023C0076071A0476061A055607C1
:100C20003A0456063A0536075A0436065A05160798
:100C30005B0416065B05F5077B04F5067B05D50707
:100C40009B04D5069B05B5077C04B5067C05950776
:100C50005C0495065C057507FB047506FB055507E6
:100C60003C0455063C0535071C0435061C051507D4
:100C7000BB041506BB051A0225001B0226001C0238
:100C80002700000C0500030C0600000C0700480AB2
:100C9000490AC6040009F1024A0AC6054F0A500A69
:100CA000070C0500BF0C06000F0C0700570A580A76
:100CB000C6045A0A5B0A05023A0006023B00070214
:100CC0003C00C605A304C305000900086300E10950
:100CD0006300B7096F00A305C305C7046F0A700A54
:100CE00087040F022A0063009709AF0263006809B6
:100CF0000A023600630068090A023500A305C3052D
:100D0000F606A00A7000010C3100A305C305050911
:100D1000A305C305B002F70CD0010306B20A1702FF
:100D200095004307830A180296004307830A0304C9
:100D30005003310071037103F101A305C3050509D7
:100D4000A305C3056505A40AA50A6504010CB20044
:100D50000307B30003066B0A8705AE0AAF0AC7058F
:100D60006300F00A2A0C2A006300970918022A007F
:100D70006300970917022A0063009709870500009E
:100D8000000000000000C7056300F00A000C050029
:100D9000000C0600000C070005023A0006023B00AA
:100DA00007023C007607DB047606DB0556071A04CB
:100DB00056061A0536073A0436063A0516075A0447
:100DC00016065A05F5075B04F5065B05D5077B0497
:100DD000D5067B05B5079B04B5069B0595077C04E6
:100DE00095067C0575071C0475061C055507BB0494
:100DF0005506BB0535073B0435063B0515071B04A7
:100E000015061B051A0225001B0226001C022700DE
:100E1000000000000000000027040009F1020D0B93
:100E20002705070C0500FF0C0600090C0700270426
:100E3000000000000000000005023A0006023B002E
:100E400007023C00A304C30533092705000863001B
:100E5000E109070C0500090C0700FF0C0600630000
:100E6000B7096F00A305C305C704360B370BA704EA
:100E70000F022A0063009709AF02630068090A02A3
:100E80003600630068090A023500A305C305F606AB
:100E9000670B7000010C3100A305C305C609A3054B
:100EA000C305B002F70CD0010306790B17029500B9
:100EB00043074A0B1802960043074A0B03045003EA
:100EC000310071037103F101A305C305C609A30530
:100ED000C30565056B0B6C0B6504010CB2000307C1
:100EE000B3000306320BA705750B760BC70563002D
:100EF000F00A2A0C2A006300970918022A006300EE
:100F0000970917022A0063009709A705000000004F
:100F100000000000C7056300F00A6D0C8A0043075B
:100F2000930B6300160B310C8A0043079B0B45059E
:100F3000A304C3058E0B320C8A004307A30B4504A0
:100F4000A304C3058E0B330C8A004307AC0B010CC2
:100F50003D00A304C3059B0B340C8A004307B40B6C
:100F60006605A304C305950B350C8A004307BC0B2B
:100F70006604A304C305950B360C8A004307C50B12
:100F8000010C3D00A304C305B30B370C8A004307D3
:100F9000CE0B080C3D00A304C3059B0B380C8A0044
:100FA0004307D70B080C3D00A304C305B30B390C52
:100FB0008A004307DE0BA304C305C10B300C8A0073
:0E0FC0004307E50BA304C305DA0B6300110B16
:020FFE00F90AEE
:081000000000050003000000E0
:021FFE00F90FD9
:00000001FF
